:1000000012C02AC029C028C027C026C025C024C0CD
:1000100023C022C021C020C01FC01EC01DC01CC0E4
:100020001BC01AC019C011241FBECFEDCDBF10E0F8
:10003000A0E6B0E0E2EFF3E002C005900D92A0363A
:10004000B107D9F710E0A0E6B0E001C01D92A036DC
:10005000B107E1F798D1CBC1D3CFDF93CF93CDB721
:10006000DEB7E7E3F0E08FEF8083A1E3B0E0E1E308
:10007000F0E0808188608C93A1E3B0E0E1E3F0E000
:10008000808184608C93E8E3F0E08FEF8083A2E3CB
:10009000B0E0E2E3F0E0808188608C93A2E3B0E01E
:1000A000E2E3F0E0808184608C931DD01CD01BD0F3
:1000B00080E33FD018D080E33CD042D180E339D0F8
:1000C00088E237D0A7E3B0E0E7E3F0E08081807F0B
:1000D0008C938CE02ED086E02CD082E02AD003D006
:1000E000CF91DF910895DF93CF930F92CDB7DEB715
:1000F00082E3898304C024D18981815089838981E5
:100100008823C9F70F90CF91DF910895DF93CF93A4
:100110000F92CDB7DEB788EC898304C0E4DF898114
:100120008150898389818823C9F70F90CF91DF910E
:100130000895DF93CF930F92CDB7DEB7898384E024
:10014000698140E004D00F90CF91DF910895DF9353
:10015000CF9300D000D00F92CDB7DEB789836A83EA
:100160004B838981282F30E03D832C838C819D81B6
:10017000843091057CF42C813D8122303105BCF422
:100180008C819D810097F9F02C813D8121303105D2
:10019000B9F020C08C819D8184309105D9F4A2E30F
:1001A000B0E0E2E3F0E08081877F8C9313C08B8125
:1001B0008F738B838981833019F48B81805C8B836F
:1001C0008B818068B6DFA2E3B0E0E2E3F0E08081FB
:1001D00088608C93A2E3B0E0E2E3F0E08081846089
:1001E0008C93A2E3B0E0E2E3F0E0808184608C9342
:1001F000A8E3B0E0E8E3F0E08081982F9F708A8167
:10020000807F892B8C93A8E3B0E0E8E3F0E0808165
:10021000982F9F708A81807F892B8C93A2E3B0E016
:10022000E2E3F0E080818B7F8C93A2E3B0E0E2E335
:10023000F0E080818B7F8C9383D0E7E3F0E08081D6
:10024000803FB9F58A818295807F8A83A2E3B0E0FE
:10025000E2E3F0E0808184608C93A2E3B0E0E2E32B
:10026000F0E0808184608C93A8E3B0E0E8E3F0E004
:100270008081982F9F708A81807F892B8C93A8E33F
:10028000B0E0E8E3F0E08081982F9F708A81807F62
:10029000892B8C93A2E3B0E0E2E3F0E080818B7FD6
:1002A0008C93A2E3B0E0E2E3F0E080818B7F8C935B
:1002B00047D00F900F900F900F900F90CF91DF913C
:1002C0000895DF93CF9300D000D00F92CDB7DEB763
:1002D0008B838B81282F30E03D832C838C819D8103
:1002E0008330910569F02C813D812430310531F056
:1002F0008C819D818230910531F006C082E0E1DF82
:1003000080E48A8301C01A828A81898307C081E0E0
:1003100060E249811CDF89818F5F89838981282F71
:1003200030E08A81882F90E00F96281739077CF3F8
:100330000F900F900F900F900F90CF91DF91089535
:10034000DF93CF9300D000D00F92CDB7DEB784E417
:10035000898302C08981898189818A838A818D8389
:100360008D81882311F081E08D839D818A81815068
:100370008983992379F70F900F900F900F900F902A
:10038000CF91DF910895DF93CF93CDB7DEB7BEDE77
:1003900064DEBCDEBBDE81E061E448E0D8DEB6DED0
:1003A000B5DE80E062E440E0D2DEB0DEAFDE80E0C9
:1003B00063E440E0CCDEAADEA9DE80E064E440E055
:1003C000C6DEA4DEA3DEE7E3F0E08FE08083E8E3AF
:1003D000F0E08FE080839ADEE8E3F0E085E0808360
:1003E00095DEE8E3F0E08AE0808390DEF0CFF894D9
:0203F000FFCF3D
:00000001FF
